:020000040000FA
:10000000830101308A007929FA00030E8301FB0085
:100010000A08FC008A010B1183160313BF0F112875
:10002000C00A83120317EC0F1628ED0A7C088A0019
:100030007B0E8300FA0E7A0E09001030F900F701EA
:10004000F801F60CF50C031C2B287408F80773084C
:10005000F7070318F80A0310F30DF40DF90B212824
:1000600008007508760403195628F701F8010130D5
:10007000F900F61B4028F90A0310F50DF60D392892
:1000800076087402031D462875087302031C4F2866
:100090007608F4027508F302031CF4030314F70D49
:1000A000F80DF60CF50CF90B40280800FF30F700AE
:1000B000F80008008B138B1B5A2874088A007308F9
:1000C00082000430831603139F0005149F13C13070
:1000D00083129F000A30F300F30B6C281F151F19C1
:1000E0006F281E080317C0000630831603139F00F5
:1000F000C730850008008312031306122821F30B72
:100100007E280608F0390338860086168728882856
:100110008612F3162821F30B8A2886168F2890283A
:1001200086122821861694289528861228210610E2
:1001300086169A289B2886122821283014210C30F4
:1001400014210630142183120313061201301421E6
:10015000F3162821F30BA92828298312031306126A
:1001600040307418F307F31715298312031306168A
:10017000C5208B17FF3903190800F30001308A00EE
:100180001521F60FB828F70AB8288B1377088A00CC
:10019000760882001030F3002730F400EF20FD08CD
:1001A000031DD3282D21E830F3000330F400EF20A5
:1001B000FD08031DDC282D216430F300F401EF203D
:1001C000FD08031DE4282D210A30F300F401EF207F
:1001D000FD08031DEC282D21303076071129FD087C
:1001E000031DFD03F801F80A7308F6027408031CE6
:1001F000740FF7020318F3287408F7077308F6075B
:100200000318F70A7803031D7E1408000F39F30062
:100210003030F3073A307302031C10290730F3071C
:100220007308831203130616F300F501730E0F39DA
:10023000F400831203130608F0397404860086164E
:10024000212922298612751A28297516730817295B
:100250004030F500F50B2A290800031DFD03F300CB
:10026000031D7E1430307E18F30720307E1CF30708
:10027000730811290008831203178C0083160C15CC
:100280008B138B1B402955308D00AA308D008C14A8
:100290008B178C1849290C1183128D0A840AF30BD1
:1002A0003A290800831603170C1483120C088000E7
:1002B0008D0A840AF30B52290800831603178C1346
:1002C00083128F0100308D0083130930F30020303A
:1002D00084003A2108000030831203178D008F013B
:1002E00083168C1383130930F300203084005221CD
:1002F000080020308B00831203130030850000308B
:100300008600003087008F308316810006309F0002
:10031000C7308500C0308600FF30870007309C0062
:100320008313203084008001840A841F932984165B
:100330008001840AF0300402031D982983171030CD
:1003400084008001840A70300402031DA1299030CA
:1003500084008001840AF0300402031DA9290430BE
:1003600083120313D100C4308316C4004030C80088
:100370004030D2007F30D400FF30DA00FF30DF00A1
:10038000FF30E400FF30E900403083120317BA0069
:100390007B206B218312031381010B118B176120CA
:1003A000831203132108003EAB002008023EAA007E
:1003B0000318AB0A00302D180138AC00F3012C08EB
:1003C000031DE7292008A0002108A100F129F30A54
:1003D0002C087302031DF1292A08A0002B08A10094
:1003E000F129831203134E1CFA292E18FA292E1410
:1003F0002D14002A831203132D104E18002A2E10DC
:1004000083120317B81F082A0313A001A1011B2A96
:10041000831203135D1F1B2A2F181B2A2F145D1B29
:10042000152AA00F1B2AA10A1B2A83120313A0035B
:10043000200F1B2AA103831203135D1B202A2F10F8
:10044000831203132108003EB1002008143EB000BF
:100450000318B10AF3013208031D332A2008A00053
:100460002108A1003D2AF30A32087302031D3D2A28
:100470003008A0003108A1003D2A00308312031388
:10048000AD180138B2002D1D4A2A33184A2A3314F8
:10049000AD14502A83120313AD102D19502A3310B6
:1004A000831203132108003EB5002008C83EB400A3
:1004B0000318B50AF3013608031D632A2008A000BB
:1004C0002108A1006D2AF30A36087302031D6D2A64
:1004D0003408A0003508A1006D2A003083120313F0
:1004E000AD190138B6002D1E7A2A37187A2A37142A
:1004F000AD15802A83120313AD112D1A802A3710EF
:100500000030831203132102B90002302002B80028
:10051000031CB9030030AD1B0138BA00F3013A08DF
:10052000031D972A2008A0002108A100A12AF30A90
:100530003A087302031DA12A3808A0003908A10057
:10054000A12A83120313CE1CAA2A3B18AA2A3B1401
:10055000AD17B02A83120313AD13CE18B02A3B1087
:100560000030831203132102BD0014302002BC00AE
:10057000031CBD03F3013E08031DC32A2008A0008D
:100580002108A100CD2AF30A3E087302031DCD2ADB
:100590003C08A0003D08A100CD2A003083120313BF
:1005A0003F180138BE00AD1EDA2A4018DA2A40147E
:1005B0003F14E02A831203133F10AD1AE02A4010C3
:1005C0000030831203132102C200C8302002C10090
:1005D000031CC203F3014308031DF32A2008A000F3
:1005E0002108A100FD2AF30A43087302031DFD2A16
:1005F0004108A0004208A100FD2A00308312031325
:10060000BF180138C3002D1F0A2B44180A2B4414AD
:10061000BF14102B83120313BF102D1B102B44107B
:10062000831203134B08F3004C08F4000030F5006C
:100630000130F60000308A00312003308A0077084C
:10064000C5007808C6000030F3000130F40045080A
:10065000F5004608F60000308A001D2003308A00AD
:100660007708C7007808C80048084C02CA00470845
:100670004B02C900031CCA032108013ECC0020081C
:10068000903ECB000318CC0AED1C492BA301A4011A
:100690005C2B831203136D1C5C2B4D185C2B4D14CB
:1006A000D71B562BA30F5C2BA40A5C2B83120313BE
:1006B000A303230F5C2BA403831203136D18612B78
:1006C0004D10831203134E1D6B2B4E1F6B2BCE1F31
:1006D0006B2B4E146E2B831203134E104E1D762B74
:1006E000CE1E762BCE1F762B2D15792B831203135E
:1006F0002D11CE1D812B4E1F812BCE1F812BCE1491
:10070000842B83120313CE10CE1D8C2BCE1E8C2B6C
:10071000CE1F8C2BAD168F2B83120313AD124E1DE3
:10072000972B4E1E972BCE1F972B2D169A2B83128D
:1007300003132D12CE1DA22B4E1EA22BCE1FA22BB9
:100740002D17A52B831203132D133F1DAB2BBF1D9C
:10075000AB2B4E15AE2B831203134E11BF1EB42BC1
:100760003F1EB42BCE15B72B83120313CE11BF1E21
:10077000BE2B4F18BE2B4F143F15C42B83120313EF
:100780003F11BF1AC42B4F1083120313BF1DCD2B73
:100790005018CD2B50143F16D32B831203133F1246
:1007A000BF19D32B501083120313871CD92BBF11F1
:1007B000DC2B83120313BF15071CE02BBF12E32BA6
:1007C00083120313BF164E19E92BCE19E92B3F13E1
:1007D000EC2B831203133F17071DF02B5113F32B40
:1007E0008312031351170317E81EF92B0313D201C9
:1007F000072C83120313BF1F072C5318072C531405
:10080000571A042CD20A072C83120313D203831223
:100810000313BF1B0C2C53103030F3001630F400C0
:10082000831203135208F3070318F40A00308A00F6
:100830005A2083120313D4008B178A110A125418FA
:10084000232C5512242C5516D418282CD512292CBB
:10085000D51654192D2C55132E2C5517D419322C6E
:10086000D612332CD61657123F1F3E2C0317B81C36
:100870003E2CD3183E2C03135817412C831203131C
:1008800058133F1F472C561C472CD8144A2C831250
:100890000313D8103F1F502C581C502C5815532CA4
:1008A000831203135811D81E572CA501652C8312EF
:1008B0000313581F652C5918652C5914CE19622C36
:1008C000A50A652C83120313A50383120313581B77
:1008D0006A2C59103030F3001630F40083120313E1
:1008E0002508F3070318F40A00308A005A208312FF
:1008F0000313DA008B178A110A125A18812C581226
:10090000822C5816DA18862CD811872CD8155A192B
:100910008B2C4E138C2C4E17DA19902CCE12912C56
:10092000CE165A1A952C4E12962C4E1604302502CD
:1009300083120313031CA02C0319A02CD816A12C7E
:10094000D812D81FA62CA601A701B92C8312031315
:10095000D81CB92C5B18B92C5B14CE19B32CA60F7C
:10096000B92CA70AB92C83120313A603260FB92C9E
:10097000A70383120313D818BE2C5B100330831215
:1009800003132702031DC62CE9302602831203132A
:10099000031DCC2CD817CD2CD81300305D1801388E
:1009A000DC00F3015C08031DDA2C2608A6002708EA
:1009B000A700E42CF30A5C087302031DE42CE83062
:1009C000A6000330A700E42CFF3083120313270294
:1009D000031DEC2CFF30260283120313031DF22C9F
:1009E0005D14F32C5D10DD1CF72CA801052D83127E
:1009F0000313581D052D5E18052D5E14DD1A022DFA
:100A0000A80A052D83120313A80383120313581990
:100A10000A2D5E103030F3001630F40083120313F9
:100A20002808F3070318F40A00308A005A208312BA
:100A30000313DF008B178A110A125F18212D5D1135
:100A4000222D5D15DF18262DDD11272DDD155F19EF
:100A50002B2D5D122C2D5D160330280283120313FB
:100A6000031D342DDD14352DDD10DD125D1321083D
:100A7000003EE1002008013EE0000318E10A0030DA
:100A8000E31A0138E200F3016208031D4C2D20082F
:100A9000A0002108A100562DF30A62087302031D6D
:100AA000562D6008A0006108A100562D8312031383
:100AB000DD1F5F2D64185F2D64146316652D83128E
:100AC00003136312DD1B652D6410003083120313C2
:100AD0002102E60001302002E500031CE60300309D
:100AE00057180138E700F3016708031D7C2D200823
:100AF000A0002108A100862DF30A67087302031DD8
:100B0000862D6508A0006608A100862D83120313B8
:100B1000631C8F2D68188F2D6814D714952D8312A0
:100B20000313D7106318952D6810831203134E1DFD
:100B30009F2DD81D9F2DCE1F9F2DDD17A22D831217
:100B40000313DD13CE1DAA2DD81DAA2DCE1FAA2D4D
:100B50006314AD2D831203136310E31CB42D6918C5
:100B6000B42D6914D716BA2D83120313D712E318C4
:100B7000BA2D691083120313631DC32D6A18C32D88
:100B80006A145717C92D8312031357136319C92DFC
:100B90006A10831203134E1DD32D581ED32DCE1F62
:100BA000D32DE314D62D83120313E310CE1DDE2DB7
:100BB000581EDE2DCE1FDE2D6315E12D831203138B
:100BC0006311E31DE82D6B18E82D6B14D715EE2D7E
:100BD00083120313D711E319EE2D6B10003083122B
:100BE00003132402031DF62D043023028312031382
:100BF000031DFC2DE315FD2DE311631B032E631A6A
:100C0000032EE312062E83120313E316F3016C087E
:100C1000031D0F2E2308A3002408A400192EF30A95
:100C20006C087302031D192E0330A3000030A400CA
:100C3000192E0030831203136D1A0138EC00E31FE4
:100C4000262E6E18262E6E146D152C2E831203136D
:100C50006D11E31B2C2E6E10FF3083120313240240
:100C6000031D342EFF30230283120313031D3A2E7B
:100C7000E3173B2EE3135719412ED718412E571077
:100C8000442E831203135714E31D4B2E6F184B2E63
:100C90006F146317512E831203136313E319512E3C
:100CA0006F1083120313E31F5A2E70185A2E7014FC
:100CB0005715602E831203135711E31B602E70101B
:100CC000831203134908F3004A08F4000230F500C8
:100CD0000030F60000308A00312006308A007708A4
:100CE000F1007808F200003046028316A1000730B8
:100CF000831245028316A000031CA1032008F30001
:100D00002108F4008030F5000030F60000308A0041
:100D10001D2006308A007708A2007808A300720818
:100D20002307A50071082207A4000318A50A0330B1
:100D30003507A700E8303407A6000318A70AF30117
:100D400083122808031DAA2E83162608A800270848
:100D5000A900C22EF30A831228087302031DB62EBF
:100D600083162A08A8002B08A900C22EF30A8312B2
:100D700028087302031DC22E83162C08A8002D0814
:100D8000A900C22E83120313270883162702AB0083
:100D90008312260883162602AA00031CAB03270829
:100DA000831227078316AD002608831226078316B1
:100DB000AC000318AD0A2808F3002908F4000A3033
:100DC000F5000030F60000308A00312006308A003D
:100DD0007708AE007808AF000A30F3000030F40066
:100DE0002E08F5002F08F60000308A001D2006307E
:100DF0008A007708B0007808B10031082902B300F2
:100E000030082802B200031CB30300302502B500ED
:100E100068302402B400031CB5038312D71A142FC0
:100E2000571B142F6D10172F831203136D14571BAC
:100E30001B2FD7131E2F83120313D717F30183160B
:100E40003808031D282F3D08B6003E08B700332F91
:100E5000F30A831638087302031D332F3908B600CE
:100E60003A08B700332F00308312031351190138A9
:100E70008316B8003E08013EBA003D08F43EB900B2
:100E80000318BA0A83126D1D4C2F83163B184C2F82
:100E90003B148312ED15532F83120313ED116D19BB
:100EA000532F83163B1083120313ED1D5E2F831601
:100EB0003C185E2F3C1483126D16652F83120313AA
:100EC0006D12ED19652F83163C107D30F300003054
:100ED000F400831203132308F5002408F600003001
:100EE0008A001D2007308A0077088316BD00780825
:100EF000BE0000304002031D7F2F08303F02031C5C
:100F00008C2F0030C0020830BF02031CC003411BFD
:100F10008B2F41178C2F411383120313ED1F932F37
:100F20008316C201A32F83160313C11FAA2F4318D0
:100F3000AA2F43148312ED1AA02F8316C20AA32FDF
:100F400083160313C20383160313421CA92F4411F3
:100F5000AA2F441583160313C11BAF2F43102D3046
:100F600083160313420283120313031DB92F6D1757
:100F7000BA2F6D13ED126D1FC42F83164518C42FA1
:100F800045148312ED17CB2F83120313ED136D1B42
:100F9000CB2F8316451083160313441FD52FC41F70
:100FA000D52FC81FD52F4617D82F831603134613E6
:100FB0005A1CE02F481FE02F4D1CE02F4714E32F51
:100FC000831603134710DA1CEB2F5A1DEB2FCD1C91
:100FD000EB2FC714EE2F83160313C710DA1DF62F5D
:100FE0005A1EF62F4D1DF62F4715F92F83160313A2
:100FF00047118A15002800000000000000000000D2
:10100000DA1E08285A1F0828CD1D0828C7150B28E6
:1010100083160313C711DA1F13285F1C13284D1EF4
:101020001328471616288316031347125F1D1E2820
:10103000DF1C1E28CD1E1E28C71621288316031369
:10104000C712DF1D29285F1E29284D1F2928471791
:101050002C28831603134713DF1E34285F1F342800
:10106000CC1C3428C717372883160313C713DF1F78
:101070003F28641C3F28CD1F3F2846144228831672
:1010800003134610E41C4A28641D4A28491C4A28B8
:10109000C6144D2883160313C610E41D5528641E7C
:1010A00055284C1C552846155828831603134611FD
:1010B000E41E6028641F6028C91C6028C6156328C8
:1010C00083160313C611E41F6B28691C6B28491D86
:1010D0006B2846166E28831603134612E91C7628E1
:1010E000691D7628C91D7628C6167928831603132C
:1010F000C612E91D8128691E8128491E81284815CC
:101100008428831603134811E91E8C28691F8C2834
:10111000C91E8C28C8148F2883160313C810E91F12
:101120009728541C9728491F972848149A288316F3
:1011300003134810D41CA228541DA228C91FA2289A
:10114000C815A52883160313C811D41DAD28541E35
:10115000AD28411CAD284816B02883160313481249
:10116000D41EB828541FB828C11CB828C816BB28DC
:1011700083160313C812461BDE284718DE28C7183B
:10118000DE284719DE28C719DE28471ADE28C71AC5
:10119000DE28471BDE28C71BDE284618DE28C618B7
:1011A000DE284619DE28C619DE28461ADE28C61AA9
:1011B000DE28C61BDE2883120512E12883120313E2
:1011C000051683164819F028C818F0284818F02882
:1011D000C819F028481AF028C81AF028C613F328AE
:1011E00083160313C6174A18F728C813F828C81718
:1011F000831203171318002983160313C913032935
:1012000083160313C9178312031793180B29831628
:10121000031349130E298316031349174B18122978
:10122000411013294114CB181729C1101829C114D2
:101230003030F3001730F4005008F3070318F40AB5
:1012400000308A005A2083160313CA008B178A15B0
:101250000A123830F3001730F4005008F30703186F
:10126000F40A00308A005A2083160313CB008B1730
:101270008A150A124E183E29C9123F29C916CE18DE
:1012800043294912442949164E194829C9114929A7
:10129000C915CE194D2949114E2949154E1A522901
:1012A000C9105329C914CE1A57294C1058294C1467
:1012B0004E1B5C2949105D294914CE1B6129CD13B1
:1012C0006229CD17F3015008031D6B290030CE00B1
:1012D0000030CF00A329F30A50087302031D7529BB
:1012E0002D30CE000030CF00A329F30A500873023E
:1012F000031D872983120317630883160313CE0087
:1013000083120317640883160313CF00A329F30A7B
:1013100050087302031D9529831249088316CE00D5
:1013200083124A088316CF00A329F30A50087302D8
:10133000031DA329831249088316CE0083124A088D
:101340008316CF00A32983160313C11EA929D00138
:10135000B72983160313411EB7295118B729511411
:101360004119B429D00AB72983160313D003831671
:101370000313411ABC295110831603134111831220
:10138000ED1FC7298316C11DC7294116CA29831617
:10139000031341120330500283160313031CD22996
:1013A000031DD429C115D529C111C112521BDC2935
:1013B000411FDF295214DF298316031352108316AD
:1013C0000313521CE729411FE729C117EA29831695
:1013D0000313C113521EEE295213F129831603136E
:1013E00052178312ED1BF9298316521DFC29D214C2
:1013F000FC2983160313D21083160313D218042A70
:10140000C119042A5212072A831603135216D21D39
:101410000E2A53180E2A53145215142A8316031336
:101420005211D219142A531000308316031350029C
:1014300083160313031C202A0319202AD216212AFB
:10144000D212C41D2B2AD21E2B2AD21F2B2A441C97
:101450002B2AC4142E2A83160313C4102A304202E6
:1014600083160313031C362A031D382AD217392A80
:10147000D2130130420283160313031C412A441481
:10148000422A44102C30420283160313031D4A2AB9
:10149000D4174B2AD413C41C532A5518532A551455
:1014A000831285165A2A8312031385128316C418D1
:1014B0005A2A551083160313441D632A5618632AAB
:1014C0005614C415692A83160313C4114419692AD2
:1014D000561083160313D41F722A5718722A5714F2
:1014E0004416782A831603134412D41B782A571003
:1014F00083160313441E802AD21E802AC416832A10
:1015000083160313C4124417C4174208D8000230CC
:101510005802031C912A0319912A44130230D8005F
:10152000982A013058020318982AC4130130D800B1
:101530005A1448174208D90004305902031CA62A3D
:101540000319A62A5A100430D900AD2A03305902D3
:101550000318AD2A48130330D900DA145A1542088B
:10156000DB0006305B02031CBB2A0319BB2ADA101E
:101570000630DB00C22A05305B020318C22A5A116A
:101580000530DB00DA155A164208DC0008305C0230
:10159000031CD02A0319D02ADA110830DC00D72A1C
:1015A00007305C020318D72A5A120730DC00DA161B
:1015B0005A174208DD000A305D02031CE52A0319B0
:1015C000E52ADA120A30DD00EC2A09305D02031840
:1015D000EC2A5A130930DD00DA175F144208DE00E6
:1015E0000C305E02031CFA2A0319FA2ADA130C30B3
:1015F000DE00012B0B305E020318012B5F100B3055
:10160000DE005F15DF144208E0000E306002031CAC
:101610000F2B03190F2B5F110E30E000162B0D302E
:1016200060020318162BDF100D30E000DF155F1687
:101630004208E10010306102031C242B0319242B03
:10164000DF111030E1002B2B0F30610203182B2B20
:101650005F120F30E100DF165F174208E200123020
:101660006202031C392B0319392BDF121230E200FE
:10167000402B113062020318402B5F131130E2003F
:10168000DF1764144208E30014306302031C4E2B7E
:1016900003194E2BDF131430E300552B1330630274
:1016A0000318552B64101330E300E414641542084A
:1016B000E50016306502031C632B0319632BE4104D
:1016C0001630E5006A2B1530650203186A2B641189
:1016D0001530E500E41564164208E600183066028D
:1016E000031C782B0319782BE4111830E6007F2BAC
:1016F0001730660203187F2B64121730E600E416D9
:1017000064174208E7001A306702031C8D2B031987
:101710008D2BE4121A30E700942B1930670203185E
:10172000942B64131930E700E41769144208E800A9
:101730001C306802031CA22B0319A22BE4131C30DB
:10174000E800A92B1B3068020318A92B69101B3075
:10175000E800E91469154208EA001E306A02031C19
:10176000B72B0319B72BE9101E30EA00BE2B1D3032
:101770006A020318BE2B69111D30EA00E9156916CB
:101780004208EB0020306B02031CCC2B0319CC2B3E
:10179000E9112030EB00D32B1F306B020318D32B41
:1017A00069121F30EB00E91669174208EC0022307D
:1017B0006C02031CE12B0319E12BE9122230EC002F
:1017C000E82B21306C020318E82B69132130EC0060
:1017D000E91754144208ED0024306D02031CF62B67
:1017E0000319F62BE9132430ED00FD2B23306D0295
:1017F0000318FD2B54102330ED00D4145415420867
:10180000EE0026306E02031C0B2C03190B2CD41097
:101810002630EE00122C25306E020318122C5411C3
:101820002530EE00D41554164208EF0028306F0220
:10183000031C202C0319202CD4112830EF00272C56
:1018400027306F020318272C54122730EF00D416CC
:10185000541742088312031790002A301002031C09
:101860003B2C03193B2C83160313D4122A3083120A
:1018700003179000462C293010020318462C8316BB
:101880000313541329308312031790008316031394
:10189000C41A4D2C83128511502C83120313851505
:1018A00003171118572C83160313CC105A2C8316C8
:1018B0000313CC14831203179118622C831603139D
:1018C0004D13652C831603134D178312031711193B
:1018D0006D2C83160313CD12702C83160313CD16B3
:1018E000831203179119782C831603134D127B2C46
:1018F000831603134D1683120317111A832C8316B4
:101900000313CD11862C83160313CD1583120317F1
:10191000911A8E2C831603134D11912C83160313E9
:101920004D1583120317111B992C83160313CD1029
:101930009C2C83160313CD1483120317911BA42C24
:10194000831603134D10A72C831603134D14F301B4
:101950005008031DB22C0030831203179100003091
:101960009200E62CF30A50087302031DBE2C0030CF
:1019700083120317910000309200E62CF30A5008FE
:101980007302031DCA2C831203175F0891006008BD
:101990009200E62CF30A50087302031DD82C831220
:1019A0004508031791000313460803179200E62C1D
:1019B000F30A50087302031DE62C8312450803172F
:1019C00091000313460803179200E62C0230831699
:1019D0000313500283120313031CF22C0319F22C7D
:1019E000D116F32CD112F30103171708031DFD2C98
:1019F00015089300160894000C2DF30A0317170816
:101A00007302031D0C2D0313230803179300031304
:101A10002408031794000C2D4030F3001730F40015
:101A2000831603130310500DF3070318F40A003054
:101A30008A005A20831203179500F30A0319F40A47
:101A400000308A005A208312031796008B178A15DC
:101A50000A1200300313D11A01380317970018181F
:101A6000452D831603134C1D452D0030F300003027
:101A7000F40000308A00AD205030F6001730F70037
:101A800000308A00B5208A150A12831603134C1DF4
:101A90004D2D831203171814502D8312031718109D
:101AA0001918662D83160313CC1D662D0030F30024
:101AB0000030F40000308A00AD206130F6001730AD
:101AC000F70000308A00B5208A150A128316031326
:101AD000CC1D6E2D831203171914712D8312031759
:101AE000191003135D1D792D83164C1E792D4C158D
:101AF0007C2D831603134C1183125D19842D8316DC
:101B00004C1E842DCC15872D83160313CC11831204
:101B100003171A18A42D831603134C1EA42D00308E
:101B2000F3000130F40000308A00AD208316031367
:101B30002E08F6002F08F7007E100230FD0000305E
:101B40008A00CA208A150A12831603134C1EAC2D74
:101B5000831203171A14AF2D831203171A101B18C0
:101B6000C52D831603134C1EC52D0430F300013020
:101B7000F40000308A00AD207230F6001730F70014
:101B800000308A00B5208A150A12831603134C1EF2
:101B9000CD2D831203171B14D02D831203171B1096
:101BA0001C18EB2D831603134C1EEB2D0530F30090
:101BB0000130F40000308A00AD2083160313320890
:101BC000F6003308F7007E100530FD0000308A0073
:101BD000CA208A150A12831603134C1EF32D831292
:101BE00003171C14F62D831203171C101D18112E39
:101BF000831603134C1E112E0630F3000130F4003F
:101C000000308A00AD20831603133608F60037082B
:101C1000F7007E140330FD0000308A00CA208A15C8
:101C20000A12831603134C1E192E831203171D1458
:101C30001C2E831203171D101E18322E8316031339
:101C40004C1E322E0930F3000130F40000308A00BF
:101C5000AD207430F6001730F70000308A00B52050
:101C60008A150A12831603134C1E3A2E8312031789
:101C70001E143D2E831203171E101F18512E251DF2
:101C8000512E0030F3000030F40000308A00AD2007
:101C90007830F6001730F70000308A00B5208A153A
:101CA0000A1283120317251D572E1F145A2E831252
:101CB00003171F1020186E2EA51C6E2E0030F30087
:101CC0000130F40000308A00AD208930F600173072
:101CD000F70000308A00B5208A150A128312031714
:101CE000A51C742E2014772E8312031720102118A0
:101CF0008B2E251C8B2E0030F3000130F4000030B9
:101D00008A00AD209A30F6001730F70000308A00C4
:101D1000B5208A150A1283120317251C912E21144F
:101D2000942E8312031721102218AA2E8316031350
:101D3000CC1FAA2E0030F3000130F40000308A00DE
:101D4000AD20AB30F6001730F70000308A00B52028
:101D50008A150A1283160313CC1FB22E831203179F
:101D60002214B52E8312031722102318CB2E8316AC
:101D700003134C1FCB2E0030F3000130F400003071
:101D80008A00AD20BC30F6001730F70000308A0022
:101D9000B5208A150A12831603134C1FD32E831203
:101DA00003172314D62E8312031723102418EC2EA6
:101DB00083160313CC1EEC2E0030F3000130F40028
:101DC00000308A00AD20CD30F6001730F70000302B
:101DD0008A00B5208A150A1283160313CC1EF42E2E
:101DE000831203172414F72E8312031724100313EE
:101DF000581EFF2E0317251DFF2EA514022F831238
:101E00000317A5100313D81D0A2F0317251D0A2F2A
:101E100025140D2F83120317251003134E1F172FA0
:101E20000317251D172F83160313CC171A2F83169C
:101E30000313CC138312CE1E242F0317251D242F2A
:101E4000831603134C17272F831603134C13831287
:101E50004E1E312F0317251D312F83160313CC1669
:101E6000342F83160313CC128312031726184A2F1C
:101E7000A51F4A2F0030F3000030F40000308A0024
:101E8000AD20DE30F6001730F70000308A00B520B4
:101E90008A150A1283120317A51F502F2614532FD9
:101EA00083120317261027186C2FA51F6C2F0030E4
:101EB000F3000130F40000308A00AD2083120317D4
:101EC0002B08F6002C08F7007E100330FD000030D0
:101ED0008A00CA208A150A1283120317A51F722FBF
:101EE0002714752F8312031727102818892FA51F71
:101EF000892F0330F3000130F40000308A00AD2058
:101F0000EF30F6001730F70000308A00B5208A1550
:101F10000A1283120317A51F8F2F2814922F8312E2
:101F2000031728102918AB2FA51FAB2F0430F3007F
:101F30000130F40000308A00AD20831203172F080F
:101F4000F6003008F7007E100530FD0000308A00F2
:101F5000CA208A150A1283120317A51FB12F29144C
:101F6000B42F8312031729102A18C82FA51FC82FB2
:101F70000530F3000130F40000308A00AD20F1306C
:101F8000F6001730F70000308A00B5208A150A12D3
:101F900083120317A51FCE2F2A14D12F83120317E4
:101FA0002A1003132608F3002708F4000A30F5006E
:101FB0000030F60000308A0031200F308A007708A8
:101FC0000317AB007808AC002B08F3002C08F400D2
:101FD0000A30F5000030F60000308A001D200F3076
:101FE0008A007708AD007808AE008A110A1600282A
:101FF00000000000000000000000000000000000E1
:102000002E08031327020317B0002D08031326021E
:102010000317AF00031CB00331182028A51D20288A
:102020000030F3000030F40000308A00AD20FD30B5
:10203000F6001730F70000308A00B5208A110A1622
:1020400083120317A51D262831142928831203178C
:10205000311032183D28251E3D280030F300013094
:10206000F40000308A00AD200E30F6001830F70082
:1020700000308A00B5208A110A1683120317251E24
:1020800043283214462883120317321033185A2873
:10209000A51E5A280030F3000130F40000308A00F9
:1020A000AD201F30F6001830F70000308A00B52050
:1020B0008A110A1683120317A51E60283314632899
:1020C00083120317331034187728251F7728003020
:1020D000F3000130F40000308A00AD203030F6000B
:1020E0001830F70000308A00B5208A110A168312D2
:1020F0000317251F7D2834148028831203173410FA
:1021000003135D1D88280317A51D882825168B2815
:102110008312031725120313DD1D93280317A51D32
:102120009328A516962883120317A51203135D1E84
:102130009E280317A51D9E282517A1288312031783
:1021400025130313561DA928D61DA92883164C163E
:10215000AC28831603134C128312D61CB428D61D48
:10216000B42803172515B728831203172511031365
:10217000561CBF28D61DBF280317A517C2288312D7
:102180000317A5130313581CCA28D61DCA28031702
:10219000A515CD2883120317A5110313561ED328A6
:1021A0000317B501DA28831203173618FD28B91E64
:1021B000FD28B50A351CDE283717DF283713B51C74
:1021C000E328B716E428B712351DE8283815E928A2
:1021D0003811B51DED28B815EE28B811351EF228B6
:1021E0003917F3283913B51EF7283816F82838128E
:1021F000351FFC283A15FD283A1183120317B91E22
:102200000329361406298312031736103B181B299D
:102210000313561F1B290C30F3000130F40000306B
:102220008A00AD204130F6001830F70000308A00F7
:10223000B5208A110A1683120313561F2229031789
:102240003B142529831203173B103C183A2903132A
:10225000D61F3A290C30F3000130F40000308A0018
:10226000AD204630F6001830F70000308A00B52067
:102270008A110A1683120313D61F412903173C142F
:102280004429831203173C10831603134C1E4F2955
:1022900083120317381C4F29031356175229831230
:1022A0000313561383164C1E5C2983120317381828
:1022B0005C290313D6175F2983120313D613051D58
:1022C000642903173810672983120317381403137E
:1022D000CE1F6F293F1F6F298316D21572298316CF
:1022E0000313D21183120317B8188129831603131D
:1022F000521F812983120317D31881290313CE1784
:10230000842983120313CE13D9302102031D8A2995
:102310003030200283120317031C922903199229DB
:10232000B8169329B812D93003132102031D9A2934
:10233000F9302002831203170318A0293817A129A6
:102340003813B81EA729381FA7293714AA298312C2
:1023500003173710B71CB1293D18B1293D14B81720
:10236000B72983120317B813B718B7293D10FF30E8
:10237000831203132102031DBF293630200283126A
:102380000317031CC7290319C7293715C829371193
:102390003718CE293719CE29B710D1298312031740
:1023A000B714371ED8293E18D8293E14B715DE2990
:1023B00083120317B711371ADE293E108312031751
:1023C000B719E7290313D719E729ED10EA29831272
:1023D0000313ED140317371DF2293F18F2293F1498
:1023E0003716F8298312031737123719F8293F10C7
:1023F0009630831203174002831203170318022A30
:10240000B717032AB7133A1C0A2A41180A2A41149B
:10241000BA15102A83120317BA113A18102A41105C
:1024200083120317BA18182AB71F1B2A3A141B2A3B
:10243000831203173A1083120317BA1D282A0313B5
:102440002918282A291401308A005D2112308A00B7
:1024500083120317BA192E2A0313291003173A1AE5
:10246000352A3A1F382ABA16382A83120317BA12A5
:1024700083120317B91B402A3A1D432A3A16432AEE
:10248000831203173A12831203173A17BA1E4C2A03
:10249000B81D4C2ABA174F2A83120317BA13BA1F52
:1024A000572A4218572A42140313D6155E2A83125C
:1024B0000313D6110317BA1B5E2A421083120317A7
:1024C000BA1C652AC301C4017A2A83160313411F6B
:1024D000BD2A831203174518BD2A4514C618742A4D
:1024E000C30F7A2AC40A7A2A83120317C303430F3D
:1024F0007A2AC40383120317431C802A4614812AB4
:102500004610C31C852A3916862A3912431D8A2A89
:10251000B9158B2AB911C31D8F2A3915902A391183
:10252000431E942AB914952AB910C31E992A391446
:102530009A2A3910431F9E2AC6179F2AC613C31F03
:10254000A32A4617A42A4613441CA82AC616A92A59
:10255000C612C41CAD2A4616AE2A4612441DB22A23
:10256000C615B32AC611C41DB72A4615B82A461186
:10257000441EBC2ABA14BD2ABA1083160313411B89
:10258000C42A83120317451083120317C6103A1A80
:10259000D12A83160313411FD12A83120317B916B8
:1025A000D42A83120317B91203135118DE2AD11843
:1025B000DE2AD119DE2A0317B913E12A8312031781
:1025C000B917381CE92A4718E92A4714031351148C
:1025D000F02A83120313511003173818F02A4710FA
:1025E000831203173818FA2A4818FA2A48140313D2
:1025F000D114012B83120313D1100317381C012BA4
:102600004810831203132108003E0317CA00031366
:102610002008013E0317C9000318CA0A0313200843
:10262000F3002108F4000230F5000030F60000301D
:102630008A00312013308A0077080317CB0078080E
:10264000CC004908F3004A08F4000230F5000030DD
:10265000F60000308A00312013308A007708CD0060
:102660007808CE004C084E02031D382B4B084D0253
:1026700083120313031D3E2B51113F2B5115511E85
:10268000482B03174F18482B4F140313D1154F2B0A
:1026900083120313D111511A4F2B03174F108312BA
:1026A00003173A19582BB91B582B031356125B2BDF
:1026B000831203135616511B612B0317D001D1014E
:1026C000762B83160313411FAA2B8312031752186C
:1026D000AA2B5214D41A702BD00F762BD10A762B3A
:1026E00083120317D003500F762BD10383120317E5
:1026F000501C7C2BD3157D2BD311D01C812B531652
:10270000822B5312501D862BD316872BD312D01D2C
:102710008B2B53178C2B5313501E902BD317912BAD
:10272000D313D01E952B5414962B5410501F9A2B54
:10273000D4149B2BD410D01F9F2B5415A02B5411B5
:10274000511CA42BD415A52BD411D11CA92B541684
:10275000AA2B541283160313411BB12B83120317A8
:10276000521083120317D31CBA2B0313511FBA2B19
:10277000BF17BD2B83120313BF13D11BC42B031729
:10278000531CC72BD314C72B83120317D3108312E8
:102790000317D31CD02B531DD02B0313D117D32BCE
:1027A00083120313D1130317531DDA2BD318DA2B1B
:1027B0005314DD2B831203175310541EE42B5518AA
:1027C000E42B55145315EA2B831203175311541A93
:1027D000EA2B551083120317D412541BF32BD41F6A
:1027E000F62BB814F62B83120317B81083120317B5
:1027F000B81C002C0313551D002C03175417032C71
:102800008312031754130313551D0B2C0317B81809
:102810000B2CD4170E2C83120317D41303133F1B56
:102820001F2C55181F2CD5181F2C0317E81B1F2C05
:10283000831614181F2C831203135112222C831297
:1028400003135116511B2B2C031756182B2C5614FF
:1028500003135514322C831203135510511F322CBD
:102860000317561083120313511F3D2C03175718DB
:102870003D2C57140313D514442C83120313D51085
:10288000511B442C0317571083120313511F4E2C56
:102890000317D3184E2C0313D515512C8312031391
:1028A000D511D51D5A2C031758185A2C5814031338
:1028B0005515612C831203135511D519612C03177B
:1028C000581083120317B8186A2CD3186A2C0313F4
:1028D00056156D2C8312031356110317B81C752C53
:1028E000D318752C0313D614782C83120313D61027
:1028F0000317D31C802C0313551F802C5814832CD2
:102900008312031358100317D31C8B2C0313D51EEB
:102910008B2C56148E2C8312031356100317D31CC2
:10292000962C0313551E962CD517992C831203133E
:10293000D5130317681CA12C0313A2010317D90197
:10294000B72C83120317E81CB72C5A18B72C5A144B
:10295000E819B02C0313A20FB72C0317D90AB72C10
:1029600083120313A203220FB72C0317D903831278
:102970000317E818BC2C5A10831203132208F30023
:1029800003175908F4005030F5000030F60000300D
:102990008A001D2014308A007708DB007808DC00EC
:1029A0005C08013EDE005B08903EDD000318DE0A95
:1029B0006608F3006708F4000030F5000130F60007
:1029C00000308A00312014308A007708DF00780850
:1029D000E0000030F3000130F4005F08F50060080B
:1029E000F60000308A001D2014308A007708E100CC
:1029F0007808E20062086702E40061086602E3000A
:102A0000031CE40303132208053E0317E5005D08D9
:102A1000F3005E08F4000430F5000030F6000030EA
:102A20008A00312015308A007708E6007808E70030
:102A300003133F1F242DD51F242D8316521F242D31
:102A400083120317E814272D83120317E810F301EC
:102A50006A08031D342D831603135008D000831217
:102A600003176908E900422DF30A6A087302031D7F
:102A7000422D023083160313D00000308312031757
:102A8000E900422D00308312031768190138EA006B
:102A9000E81C4F2D6B184F2D6B146815552D8312A4
:102AA00003176811E818552D6B1083120317EE18E1
:102AB000632D6E186F2D0313CE1D6F2D0317EC01C0
:102AC000ED01EE14E8150030831203176D02031DAB
:102AD0006B2D10306C02031C6F2DEE10E811831269
:102AE0000313CE1D762D03176E14792D8312031751
:102AF0006E1023300313220283120317031C842D4C
:102B00000319842D6814852D6810681A8D2D031300
:102B1000D61A8D2D0317E812902D83120317E8168D
:102B2000D31C972D6F18972D6F1468169D2D831247
:102B300003176812D3189D2D6F10831603171018F2
:102B4000B42D8312681FB42D0030F3000030F40060
:102B500000308A00AD204B30F6001830F70000300E
:102B60008A00B5208A110A1683120317681FBB2D2D
:102B700083161014BE2D8316031710101118D72DAD
:102B80008312681FD72D0030F3000130F4000030AD
:102B90008A00AD20831203176508F600F7017E1046
:102BA0000230FD0000308A00DC208A110A168312F0
:102BB0000317681FDE2D83161114E12D83160317EA
:102BC00011101218F62D8312681FF62D0230F30033
:102BD0000130F40000308A00AD205C30F60018307F
:102BE000F70000308A00B5208A110A1683120317F5
:102BF000681FFD2D83161214002E83160317121062
:102C000083120313D51F092ED61D092E031768172B
:102C10000C2E831203176813D318152E831613185E
:102C2000152E13148312E8171C2E83120317E813B2
:102C3000D31C1C2E8316131083120317D31C262EAD
:102C400083161518262E151414142E2E831603170A
:102C500014108312D3182E2E831615100A12CF29A2
:102C600001340234043408341034203440348034C5
:102C7000083409340A340B340C340D340E340F3458
:102C80001034113412341334143415341634173408
:102C9000183419341A341B341C341D341E341F34B8
:102CA0002034213422342334243425342634273468
:102CB000283429342A342B342C342D342E342F3418
:102CC00030343134323433343434353436343734C8
:102CD000383439343A343B343C343D343E343F3478
:102CE0004034413442344334443445344634473428
:102CF000483449344A344B344C344D344E344F34D8
:102D00005034513452345334543455345634573487
:102D1000583459345A345B345C345D345E345F3437
:102D200060346134623463346434653466346734E7
:102D3000683469346A346B346C346D346E346F3497
:102D40007034713472347334743475347634773447
:102D5000783479347A347B347C347D347E347F34F7
:102D600080348134823483348434853486348734A7
:102D7000883489348A348B348C348D348E348F3457
:102D80009034913492349334943495349634973407
:102D9000983499349A349B349C349D349E349F34B7
:102DA000A034A134A234A334A434A534A634A73467
:102DB000A834A934AA34AB34AC34AD34AE34AF3417
:102DC000B034B134B234B334B434B534B634B734C7
:102DD000B834B934BA34BB34BC34BD34BE34BF3477
:102DE000C034C134C234C334C434C534C634C73427
:102DF000C834C934CA34CB34CC34CD34CE34CF34D7
:102E0000D034D134D234D334D434D534D634D73486
:102E1000D834D934DA34DB34DC34DD34DE34DF3436
:102E2000E034E134E234E334E434E534E634E734E6
:102E3000E834E934EA34EB34EC34ED34EE34EF3496
:102E4000F034F134F234F334F434F534F634F73446
:102E5000F834F934FA34FB34FC34FD34FE34FF34F6
:102E6000003400340134013401346134613461349C
:102E700000340134003402340234023402340234A7
:102E800000340034003400340034003400340034A2
:102E9000043400340534003406340034073400347C
:102EA000563443344F3420346634723465346B34D2
:102EB000763465346E3463346934613420342034BC
:102EC000003456346534743465346C3420346634DC
:102ED000723465346B34763465346E3463346934FB
:102EE000613400342E3400344D3448347A340034A4
:102EF0004634723465346B34763465346E346334FE
:102F00006934613420346C3465347034653473341E
:102F10000034313432342C3435346B3448347A3420
:102F20002034203420342034203420342034203401
:102F30002034003420342034353430346B34483479
:102F40007A34203420342034203420342034203487
:102F500020342034003420343134303430346B3475
:102F600048347A342034203420342034203420343F
:102F700020342034203400342034203420343134C0
:102F80004D3448347A3420342034203420342034F2
:102F900020342034203420340034203420343134A0
:102FA00030344D3448347A342034203420342034C2
:102FB0002034203420342034203400344B34463440
:102FC00020346634723465346B34763465346E3450
:102FD00063346934613420342034203400342E3496
:102FE00000344D3448347A342034203420342034B2
:102FF0002034203420342034003446347234653494
:103000006B3476342E3420346B3469346A3465344E
:103010006C347A3465347334203400345634433499
:103020004F342034203420342034203420342034D1
:1030300020342034203420342034203400345634DA
:1030400043344F342D344B34463420342034203430
:1030500020342034203420342034203420340034F0
:10306000563443344F342B344B34463420342034DC
:1030700020342034203420342034203420342034B0
:1030800000344C346F3463346B34003420342034D7
:10309000203420340034523465346634653472345C
:1030A00065346E3463346934613420344F345334BE
:1030B00043342034203400344D3448347A342034BE
:1030C0002034203420342034203420342034203460
:0630D0002034203400341E
:084000000000010000000000B7
:02400E003A3F37
:1042000000000000000000000000000000000000AE
:10421000000000000000000000000000000000009E
:10422000000000000000000000000000000000008E
:10423000000000000000000000000000000000007E
:10424000000000000000000000000000000000006E
:10425000000000000000000000000000000000005E
:10426000000000000000000000000000000000004E
:10427000000000000000000000000000000000003E
:10428000000000000000000000000000000000002E
:10429000000000000000000000000000000000001E
:1042A000000000000000000000000000000000000E
:1042B00000000000000000000000000000000000FE
:1042C00000000000000000000000000000000000EE
:1042D00000000000000000000000000000000000DE
:1042E00000000000000000000000000000000000CE
:1042F00000000000000000000000000000000000BE
:1043000000000000000000000000000000000000AD
:10431000000000000000000000000000000000009D
:10432000000000000000000000000000000000008D
:10433000000000000000000000000000000000007D
:10434000000000000000000000000000000000006D
:10435000000000000000000000000000000000005D
:10436000000000000000000000000000000000004D
:10437000000000000000000000000000000000003D
:10438000000000000000000000000000000000002D
:10439000000000000000000000000000000000001D
:1043A000000000000000000000000000000000000D
:1043B00000000000000000000000000000000000FD
:1043C00000000000000000000000000000000000ED
:1043D00000000000000000000000000000000000DD
:1043E00000000000000000000000000000000000CD
:1043F00000000000000000000000000000000000BD
:00000001FF
